:1000000054220D30840052280B1D09009000030E6D
:100010008F008312851D0E2891011328110F910066
:100020004220FF309C00051E172892011C28120F49
:1000300092004220FF309C00061C202893012428B7
:10004000061C130F930042201A081B0403192D28C5
:100050009B0F2D289A0F2D289D161708031D970317
:10006000180A031936281808031D98031C080319D9
:100070003C289C0B3C281D170F0E8300900E100E81
:100080000B110900FB309A00B4309B000800820776
:10009000583400344C340034203400344D34483467
:1000A0007A34003443308C008001840A8C0B54284D
:1000B0000130C10083161C308500033086000430F7
:1000C000810083128101A0308B00FE3086001C214C
:1000D0007D2242209D128F30F5200230FB208920A6
:1000E0009D1A69281D1789228E30F52000301E1FA9
:1000F0007A280430FB2023303F225C2225304D2219
:10010000382227304D222B2223304622DC209B2010
:1001100070288A30F5200630FB2008004D229428F4
:100120003F225C22B001B10138224F30B000B03024
:10013000B1002B2208009D102E09C039031DA728ED
:100140009D14AE09AF090130AF070318AE0A2208AB
:10015000AD000310AD0DAD0DAD072D08AD000310C2
:10016000AD0DAD0DAD072D08AD000310AD0DAD0DFE
:10017000AD07F4219C218030F5203830840009300F
:100180008C000008EB20840A8C0BC1287930F52004
:100190000008EB2008003F228030AE065C22813050
:1001A000B0009030B1002B227E30B0007030B10032
:1001B00038228030AE060800562123303F222030FE
:1001C000462229304D221422322120303F220800BD
:1001D000EA20EA202030A000A10086150429013081
:1001E000F5201830552208008130A000A1008611AA
:1001F0000421861508009F004720FF3903190800D5
:10020000EB201F08013EFB28831601308600831275
:100210000615F030A00506080E39200486000611E8
:100220000615A10EF030A10506080E39210486003E
:1002300006114B309821080086012D212D212D21FA
:1002400028308600061154222830F5200830F52089
:10025000EF200630F5200C30F52854223830860087
:10026000061108001D129D1576224B30B00000309B
:10027000B10038224E30B0002030B1002B222B309C
:100280004D222222031953292B3046227D21C230D0
:100290006F212E086F212F086F218E306F210030C3
:1002A0006F2182211E131D1A9D1108001E1F5A293D
:1002B00018086C217D21C3306F2108308C009721F4
:1002C00085149721050C9E0D85108C0B5F299321B9
:1002D000892182211E1B6C216E30980008009F002E
:1002E00008308C009F0D03189321031C8E21892157
:1002F0008C0B722993218921080085149321972161
:100300008E218B298E219721851497219321972166
:100310000800972185149721851008000510831681
:1003200005108312080083160514831208000F308D
:100330008D008D0B99290800031018308C00B9012D
:10034000BB01BD01C001B60DB50DB40DC00DBD0D95
:10035000BB0DB90D8C0BCF29400EBF003D0EBC006C
:100360003B0EBA00390EB8001D103830E421393088
:10037000E4213A30E4213B30E4213C30E4211D14F7
:100380003D30E421A530BE003F30E4214030E4217F
:100390009D1C0800370884002D3080000800403084
:1003A000D8213D30D8213B30D8213930D821A3295C
:1003B0008400033000079F009F1980003030000741
:1003C0009F009F1B8000080084000F300005031968
:1003D000ED29303E80001D1408001D18E929203049
:1003E00080000408B7000800B6012E08B4002F08EA
:1003F000B50008308C00AD0C0318032A8C0BFB29C8
:10040000B401B501080003100E2AAD0C031C0E2A1E
:100410002F08B5072E0803182E0FB407B40CB50C1F
:10042000B60C8C0B052A08003108AF0730080318FA
:10043000300FAE0708003108AF023008031C300F40
:10044000AE02080031082F029F003008031C300A5A
:100450002E021F0408003008B2003108B30001303A
:10046000B1070318B00A2222031C080032303C2ACC
:1004700022220318080030303F221D160800840095
:100480000008AE00840A0008AF00080084002E08AF
:100490008000840A2F088000080084000008B00053
:1004A000840A0008B100080076308D008E018E0BA2
:1004B000572A8D0B572A0800B001AE221D19CC22F5
:1004C0004108C200C20B652A692AC20B682A6B2A3E
:1004D0006D2A01306F2A50306F2A08306F2AB10020
:1004E000B8221D191422C2221D191B222E09C0393F
:1004F000031D0800AE01AF0108008901223084000D
:1005000009308C009C228000890A840A8C0B822A84
:1005100008001D1F08001D138901223084000930C6
:100520008C009C2200020319972A0008A122890A44
:10053000840A8C0B912A0800831608148312080879
:100540000800880083160812081555308900AA3063
:1005500089008814081EAA2A8312080016081302AC
:100560000318B42A1D15B52A1D111308960008009A
:10057000140811020318BE2A1D15BF2A1D111108E7
:1005800094000800150812020318C82A1D15C92A6C
:100590001D11120895000800C10B08000330C100AE
:0205A000080051
:02400E00FA3F77
:1042000001004B0028004B0000004C004000000063
:024210000000AC
:00000001FF
